:020000020000FC
:1000000012C0189518951895189518951895189563
:100010002BC637C6189518951895189518951895E4
:100020001895189518950FE50DBF04E00EBF08E868
:1000300001BF0FEC08BB0CE207BB0EE304BB00E002
:1000400005BB0AEF01BB05E002BB00EC07B907E006
:1000500006B90AEFDCD5919A949A002700936000C4
:10006000939A06B3037C10B31470012B013CC9F4BE
:1000700005E0CDD506B3037C10B31470012B013C11
:1000800081F406B3037C10B31470012B073CC9F74D
:1000900001E000937700002700937C0000937D002F
:1000A00030C0E0E0F0E0C9D510937700E1E0F0E087
:1000B000C4D510937C00E2E0F0E0BFD510937D0042
:1000C000E3E0F0E0BAD510937E00E4E0F0E0B5D5CF
:1000D00010937F00E5E0F0E0B0D510937800E6E003
:1000E000F0E0ABD510937900E7E0F0E0A6D51093EF
:1000F0007A00E9E0F0E0A1D5133008F01127109361
:100100006000E8E0F0E099D51B3818F4123108F0EF
:1001100001C012E41093A3020AE00093A80200E0D9
:100120000093A7020093A0020093A1020093A202F1
:100130000093A90206B3037C10B31470012B073C93
:10014000C9F704E009BF02E50DB92AE023D52A95D5
:10015000E9F7C29800E000936D0000E000936E00A4
:1001600000E000936F0000E00093700000E0009357
:1001700071001AD51F3F59F0113019F00AE03FD530
:10018000F8CF01E000936D000FD51130E9F3C29A6A
:1001900000E50DB9709A1F3F19F401E0002EFEC072
:1001A000E0D3112319F002E0002EF8C00FEF7CD34A
:1001B000112319F403E0002EF1C010937600009192
:1001C0007700002319F401E0009377006DD30091CC
:1001D0009C0010917800011761F400919D0010912E
:1001E0007900011731F400919E0010917A000117F7
:1001F00041F001E000937700112710937C001093E9
:100200007D0073D2FF93EF93EC52F140EF91FF9199
:1002100010F005E023C0FF93EF93E851F140EF9118
:10022000FF9110F004E01AC0FF93EF93E450F14007
:10023000EF91FF9110F003E011C0FF93EF93E05FA7
:10024000F040EF91FF9110F002E008C0FF93EF93B0
:10025000EC5DF040EF91FF9160F001E0002E93988B
:1002600006E9D5D4939A06E9D2D40A94C1F740910D
:10027000A50200E00DBD00E00CBD03E00EBD7894CA
:100280000091770010917600101752F401E000936E
:100290007700473429F03091600031300AF436C0DD
:1002A0008BD0F89400E00EBD112399F01AF404E00D
:1002B000002E74C011241394012C6DD24091A5021C
:1002C000473459F04738A1F0433C01F100917700E1
:1002D000E7CF00916000023029F00091770003958C
:1002E00000937700112710937C0010937D0089CF35
:1002F000009177000A9511F4009176000093770041
:10030000112710937C0010937D007BCFF89400910F
:100310007700E0E0F0E085D40A2DE1E0F0E081D460
:100320000B2DE2E0F0E07DD4009168000395031905
:100330001127080D911EE3E0F0E073D4092DE4E0ED
:10034000F0E06FD400917800E5E0F0E06AD400912D
:100350007900E6E0F0E065D400917A00E7E0F0E0B3
:1003600060D40091A302E8E0F0E05BD4009160006B
:10037000E9E0F0E056D400E010E020E1E1D108EC43
:1003800046D4939806B3037C10B31470012B073C3A
:10039000C9F70AEF3CD494989198FFCFF8941124B0
:1003A0001394F9D1E8CFC0E0D0E0E0E6FCE0DFD183
:1003B0002196D230D1F7089577D2009177000117B6
:1003C00011F01FEF0895C0909C00D0909D00E09028
:1003D0009E00F0909F00FF2011F017EF0895C0924B
:1003E0007800D0927900E0927A00A0909A00B090C4
:1003F0009B0022271E2D0D2D1695079508F421E050
:10040000802E912E6C2C722E30906800A0909A0055
:10041000B0909B0000917C0010917D002227202B42
:10042000212B49F4A0927C00B0927D0080927E0046
:1004300090927F0006C0A02EB12E80907E009090FA
:100440007F000A2D0B210F3F29F0BB2029F402E089
:10045000A01610F41EEF0895B4D152D100270093D6
:10046000A6020093A40201E01127801A910A08F461
:1004700041C0F0926E00E0926F00D0927000C09286
:1004800071005FD30FEF8CD3C0E0D0E080990FC034
:100490006DD04423DAF33FB10FEF0FB92196D2307C
:1004A00019F0779BFECFF7CF6AD3142F08953FB191
:1004B0000FEF0FB9AC9A48E0330F10F4A99A02C0BD
:1004C000A9980000AD9A4A95AD98AC98A9F72196E5
:1004D000D230E1F654D33A9431F002E01127D00E35
:1004E000E11EF11EC0CF84D1A42CB52C3090680041
:1004F00068D1B9CF062D072911F411270895F0927C
:100500006E00E0926F00D0927000C092710019D31B
:100510000FEF46D3C0E0D0E080990FC027D044232E
:10052000DAF33FB10FEF0FB92196D23019F0779B74
:10053000FECFF7CF24D3142F08953FB10FEF0FB99B
:10054000C615D70568F4AC9A48E0330F10F4A99AA1
:1005500002C0A9980000AD9A4A95AD98AC98A9F749
:100560002196D230C9F60BD311270895F89400E0F4
:100570000EBDE091A702F091A802319729F0E09317
:10058000A702F093A80220C000E00093A7020AE0AF
:100590000093A802AAD0FF93EF93E85CF040EF919C
:1005A000FF9190F401E033D3A0D0FF93EF93E85C88
:1005B000F040EF91FF9140F40AE0002E1124EBD0BF
:1005C00003EC0093A50243C003E021D336B3337C90
:1005D00020B32470322B373C21F00091A402031782
:1005E00031F03093A40200270093A6022EC0309170
:1005F000A6023395393119F03093A60226C0009334
:10060000A50233273093A4023093A602053C39F4A7
:100610001091A3021450123198F412E111C0063C5B
:1006200039F41091A3021C5F1A3850F01AE808C080
:10063000073411F441E00CC0073891F442E008C0DF
:100640001093A3020BE0212F7BD04FEF01C043E0BA
:1006500000E00DBD00E00CBD789403E00EBD0895F0
:10066000033C99F708ECD3D236B3337C20B3247023
:10067000322B333C61F306E4CAD200E002BF01E052
:1006800009BF05E003BF789436B3337C20B32470F0
:10069000322B353C99F404E6BAD236B3337C20B31E
:1006A0002470322B353C51F4009160000A950AF415
:1006B00002E00093600044274093A90236B3337CE4
:1006C00020B32470322B333CF9F602E3A0D236B3C8
:1006D000337C20B32470322B333CB1F6939AF894D8
:1006E00000E003BF04E009BFB0CF379A349A369ACE
:1006F000349BFECFE4B1F5B13798F695E7950895B0
:10070000849805E084D2849A00E010E024E018D0B8
:1007100001E07DD2809BF4CF00E010E020E010D01B
:1007200003E01BE927EF0CD00BE01091A302212F6F
:1007300007D0E0E6FCE01BD0E0E6FCE018D008952E
:10074000AB9832E008D0302F06D0312F04D0322FB2
:1007500002D0AB9A089548E0330F10F4A99A02C072
:10076000A9980000AA9A4A95AA98B1F7089558E066
:10077000809BFECF3591AC9A48E0330F10F4A99AD4
:1007800002C0A9980000AD9A4A95AD98AC98A9F717
:100790005A9571F70895B4DF112019F0E8E4FCE0F0
:1007A00002C0E0E5FCE0E3DF04E631D2E8E5FCE08E
:1007B000DEDF0EE12CD20A9479F7E8E5FCE0D7DF22
:1007C0000895CC24D0906200E0906300F090640023
:1007D0000A2D1B2D025010402227039DD00CE11C36
:1007E000F21E139DE00CF11CDD0CEE1CFF1C0895A5
:1007F00000271091690020916A003327110F221FF2
:10080000331FCA2CDB2CEE24CC0CDD1CEE1CFF2489
:100810000C0D1D1D2E1D3F1DEFEFF1E0E023F12318
:10082000E056FF4F00271E7FC090A002D090A1028B
:10083000E090A202C11621F4D21611F4E31671F071
:1008400030936E0020936F0010937000009371003E
:1008500010D0112319F044245524089501911081DA
:100860001F3F21F4083F12F00FEF1FEF402E512ED3
:10087000089567D1112309F00895A0EAB0E08AD164
:100880001D93A03AE1F7B230D1F779D130916E00E3
:1008900020916F00109170001093A0022093A1028C
:1008A0003093A20211270895402F5527CC24D090D1
:1008B0006600E0906700FF24DD0CEE1CFF1CF09248
:1008C0006E00E0926F00D0927000C0927100A09014
:1008D0006B00B0906C00EE27FF27EA15FB05FAF5D8
:1008E00030D1112311F0152F089560E1A0E8B0E098
:1008F000C0EAD0E04FD11D93AC17BD07D9F70091E6
:100900008000002359F1053EC9F000919A00109132
:100910009B00012B99F000918B00087179F40091F4
:1009200088000D3459F400918900003539F40091A4
:100930008A00033319F453954A9581F031966A95EC
:10094000A9F61DD102E01127D00EE11EF11EF09292
:100950006E00E0926F00D0927000BFCF10D1152FC3
:10096000089500E00093720000E00093730001E03E
:10097000009374000EEB00937500B4D020908800B3
:10098000309089000027122D232D3327110F221FAD
:10099000331F309372002093730010937400009300
:1009A0007500A0D000918B0010918C001F930F93C5
:1009B000005012400F911F9111F012E00895009124
:1009C0008D000093680000918E0010918F00020D41
:1009D000131D0093690010936A000091910010911B
:1009E000920000936B0010936C00A0909600B09062
:1009F0009700AA2021F4BB2011F411E00895209162
:100A00009000A29E112D002DB29E100D2091690024
:100A100030916A00020F131F009366001093670065
:100A200000916B0010916C001295212F207F1F7098
:100A30003FE0302302950F70022B332311F00F5F3C
:100A40001F4F209166003091670000241124200F71
:100A5000311F011C209362003093630000926400F8
:100A60001092650000919300109194002227332783
:100A7000FF24F12AF02AB1F400E2FF24220C331CF7
:100A8000FF1CF09272003092730020927400009369
:100A9000750028D000918000109181002091820083
:100AA00030918300D0906900E0906A00FF240D1916
:100AB0001E092F093F09442750916800652F529560
:100AC000507F62956F707727041715072607370741
:100AD00012F001E003C0002713E0089500936100C5
:100AE00011270895F0907200E0907300D090740088
:100AF000C09075003F2D2E2D1EEF1D210027309335
:100B00006E0020936F00109370000093710019D055
:100B1000112309F008952C2D31E03D21CC27DD274C
:100B2000A0E8B0E0E0EAF0E035D0C217D30722F049
:100B3000AE17BF070AF41D932196D230A9F71FD034
:100B4000089534E6C29801E100936D002DD0112381
:100B500051F4A0E0B0E11ED01E3F11F4112708951A
:100B60001197C9F704C01E3F11F411270895C29AC6
:100B700004E145D03A9509F0E5CF11E008950AD097
:100B800009D0C0E0D8E006D01F3F11F02197D9F777
:100B9000C29A08950FEF0FB9779BFECF1FB108954A
:100BA0000FB9779BFECF0895C0E0D8E0F3DF1F3F79
:100BB00021F02197D9F711E0089500916D00102FD1
:100BC0000064EEDF00916E00EBDF00916F00E8DF64
:100BD00000917000E5DF00917100E2DF112311F454
:100BE00005E901C001E0DCDFC0E0D8E0D3DF1E3F53
:100BF00029F020E8212311F02197C1F70895000082
:100C000000000000000000000A95C9F708951DE7E4
:100C10002FE000002A95E9F71A95D1F70A95B9F760
:100C200008950BD0011709F40895E199FECFFFBB99
:100C3000EEBB0DBBE29AE19A0895E199FECFFFBBAE
:100C4000EEBBE09A1DB3089553EF6E310000000033
:100C500053EF6E3500000000457869740000000015
:100C600000000000000000000FE50DBF04E00EBF13
:100C700000917700112710937C0010937D007894E9
:100C80000FCB0FB6E0916000F5E0EA9512F0FF0F90
:100C9000FCCF4091A90243954F1731F44427939913
:100CA00002C0939A01C093984093A9020FBE189571
:00000001FF
